S0220000687474703A2F2F737265636F72642E736F75726365666F7267652E6E65742F1D
S12300000C9438000C94FC240C94D51C0C9463000C9463000C9463000C9463000C946300A4
S12300200C9463000C9469250C9463000C940E290C9463000C94DC1D0C94A61D0C94731C83
S12300400C94432A0C9463000C948D290C9463000C94EB2A0C94B32A0C9463000C946300FB
S12300600C9463000C9463000C9463000C94630011241FBECFEFD0E1DEBFCDBF259A2D9A40
S1230080249A2C9A14BEA89588E10FB6F89480936000109260000FBE13E0A0E0B1E0E4E7FE
S12300A0F9E502C005900D92A43EB107D9F718E0A4EEB3E001C01D92A033B107E1F70E946C
S12300C071130C94B82C0C9400009C01F999FECF32BD21BDF89A80B508959C01F999FECF4B
S12300E01FBA32BD21BD60BD0FB6F894FA9AF99A0FBE089520E030E0F999FECF28593D4FDB
S123010032BD21BD28563240F89A80B5F901E15EF94F80832F5F3F4F81E02034380761F76B
S123012020E030E0F999FECF28573E4F32BD21BD28583140F89A80B5F901E25CFE4F808333
S12301402F5F3F4F2530310569F712BC11BC089580E090E0FC01E15EF94FE081F999FECF48
S12301601FBA88599D4F92BD81BDE0BD0FB6F894FA9AF99A0FBE8756924021E08034920769
S123018049F712BC11BC0895319B17C020E030E0F999FECF205F3F4F32BD21BD2051304016
S12301A0F89A80B5F901E455FB4F80832F5F3F4F81E02034380761F716C020E030E0F99914
S12301C0FECF205B3A4F32BD21BD20553540F89A80B5F901E455FB4F80832F5F3F4F81E0CF
S12301E02034380761F712BC11BC0895319B18C080E090E0FC01E455FB4FE081F999FECF24
S12302001FBA409692BD81BDE0BD0FB6F894FA9AF99A0FBE0F9721E08034920759F719C09F
S123022080E090E0FC01E455FB4FE081F999FECF1FBA805B9A4F92BD81BDE0BD0FB6F89492
S1230240FA9AF99A0FBE8F54954021E08034920749F712BC11BC089520E430E0F999FECFB5
S1230260205B3E4F32BD21BD20553140F89A80B5F901EB5BFE4F80832F5F3F4F203A3105BC
S123028069F712BC11BC089580E490E0FC01EB5BFE4FE081F999FECF1FBA805B9E4F92BDAE
S12302A081BDE0BD0FB6F894FA9AF99A0FBE8F549140803A910551F712BC11BC0895F99904
S12302C0FECF82E090E092BD81BDF89A80B590E09093200180931F0140911F01509120014D
S12302E0F999FECF83E090E092BD81BDF89A20B5922F80E0840F951F9093200180931F01F5
S1230300F999FECF8DEE93E092BD81BDF89A80B590E0909324018093230140912301509173
S12303202401F999FECF8EEE93E092BD81BDF89A20B5922F80E0840F951F9093240180938F
S1230340230180911F01909120019093220180932101F999FECF84E090E092BD81BDF89A35
S123036080B590E090932601809325014091250150912601F999FECF85E090E092BD81BD91
S1230380F89A20B5922F80E0840F951F9093260180932501F999FECF86E090E092BD81BD45
S12303A0F89A80B590E090930101809300014091000150910101F999FECF87E090E092BD8F
S12303C081BDF89A20B5922F80E0840F951F9093010180930001F999FECF81E090E092BD54
S12303E081BDF89A80B58093E503F999FECF88E090E092BD81BDF89A80B580931301F999B5
S1230400FECF89E591E092BD81BDF89A80B580932F01F999FECF82E094E092BD81BDF89A41
S123042090B5892F8150853078F080912F01843039F481E08093180183E68093F10506C0E6
S123044082E08093180102C090931801F999FECF89E090E092BD81BDF89A80B5809312015A
S1230460F999FECF8EE090E092BD81BDF89A80B580932801F999FECF8BE090E092BD81BDE4
S1230480F89A80B520911801829FC001112490931A0180931901F999FECF83E094E092BDC0
S12304A081BDF89A80B580931B01F999FECF8CE090E092BD81BDF89A80B520911801829F8A
S12304C0C001112490931D0180931C01F999FECF8FE691E092BD81BDF89A80B580931E01E6
S12304E0F999FECF82EF91E092BD81BDF89A80B580935A0480915A04882319F081E080935B
S12305005A04F999FECF8DE090E092BD81BDF89A80B526E0829FC001112490931501809380
S12305201401F999FECF81E791E092BD81BDF89A80B580931506F999FECF80E791E092BD62
S123054081BDF89A80B58093130685E0809384078AE080938207F999FECF8FE891E092BDC7
S123056081BDF89A80B580933001F999FECF84EF91E092BD81BDF89A80B590E02CE231E008
S1230580AC01429FC001439F900D529F900D11249093AB048093AA04F999FECF85EF91E0EF
S12305A092BD81BDF89A80B58093A704F999FECF86EF91E092BD81BDF89A80B58093A504D0
S12305C0F999FECF87EF91E092BD81BDF89A80B58093A404F999FECF88EF91E092BD81BDEE
S12305E0F89A80B590E09093A3048093A2044091A2045091A304F999FECF89EF91E092BDA7
S123060081BDF89A20B5922F80E0840F951F9093A3048093A204F999FECF8BEF91E092BDAD
S123062081BDF89A80B590E090933201809331014091310150913201F999FECF8CEF91E044
S123064092BD81BDF89A20B5922F80E0840F951F9093320180933101F999FECF8DEF91E053
S123066092BD81BDF89A80B590E090933401809333014091330150913401F999FECF8EEF1C
S123068091E092BD81BDF89A20B5922F80E0840F951F9093340180933301F999FECF8FEF0D
S12306A091E092BD81BDF89A80B590E090937803809377034091770350917803F999FECFD0
S12306C080E092E092BD81BDF89A20B5922F80E0840F951F909378038093770320E030E0AD
S12306E0F999FECF225A3E4F32BD21BD2E553140F89A80B5F901EB51FE4F8083F999FECF21
S12307002E583E4F32BD21BD22573140F89A80B5F901EE50FA4F8083F999FECF24583E4F58
S123072032BD21BD2C573140F89A80B5F901EE50FA4F808B2F5F3F4F2A30310509F0D0CF5D
S1230740F999FECF87E092E092BD81BDF89A80B580933901F999FECF83E092E092BD81BDFB
S1230760F89A80B580933A0120E030E094E6F901EF59F84F908BF999FECF245E3D4F32BDD6
S123078021BD2C513240F89A80B5F901EF59F84F80832F5F3F4F2031310549F720E030E042
S12307A0F999FECF27593E4F32BD21BD29563140F89A80B5F901E65DFE4F80832F5F3F4F9C
S12307C02430310569F720E030E0F999FECF225D3D4F32BD21BD2E523240F89A80B5F90131
S12307E0E854FC4F80832F5F3F4F2031310569F7F999FECF8DE691E092BD81BDF89A80B5D1
S123080080932701F999FECF81EF91E092BD81BDF89A80B580935904F999FECF80EF91E056
S123082092BD81BDF89A80B580932E01F999FECF86E092E092BD81BDF89A80B58093290156
S123084020E030E0F999FECF2A543C4F32BD21BD265B3340F89A80B5F901E151FE4F808318
S12308602F5F3F4F2031310569F7F999FECF87EC93E092BD81BDF89A80B580933C01F999F6
S1230880FECF88EC93E092BD81BDF89A80B580933D01F999FECF84ED93E092BD81BDF89A99
S12308A080B580936504F999FECF85ED93E092BD81BDF89A80B580936604F999FECF86ED9C
S12308C093E092BD81BDF89A80B580936704F999FECF87ED93E092BD81BDF89A80B5809322
S12308E06804F999FECF88EE93E092BD81BDF89A80B590E0909336018093350140913501D2
S123090050913601F999FECF89EE93E092BD81BDF89A20B5922F80E0840F951F90933601BC
S123092080933501F999FECF8AEE93E092BD81BDF89A80B580935C04F999FECF8CE094E01A
S123094092BD81BDF89A80B580939307F999FECF8DE094E092BD81BDF89A80B58093A00744
S1230960F999FECF8EE094E092BD81BDF89A80B580938907F999FECF8FE094E092BD81BD6C
S1230980F89A80B58093870712BC11BC089520911F0130912001F999FECF1FBA82E090E0F6
S12309A092BD81BD20BD0FB6F894FA9AF99A0FBE20911F0130912001F999FECF1FBA83E036
S12309C090E092BD81BD30BD0FB6F894FA9AF99A0FBE2091250130912601F999FECF1FBAED
S12309E084E090E092BD81BD20BD0FB6F894FA9AF99A0FBE2091250130912601F999FECF52
S1230A001FBA85E090E092BD81BD30BD0FB6F894FA9AF99A0FBE2091000130910101F9995E
S1230A20FECF1FBA86E090E092BD81BD20BD0FB6F894FA9AF99A0FBE209100013091010112
S1230A40F999FECF1FBA87E090E092BD81BD30BD0FB6F894FA9AF99A0FBE20911301F9996D
S1230A60FECF1FBA88E090E092BD81BD20BD0FB6F894FA9AF99A0FBE20911201F999FECF22
S1230A801FBA89E090E092BD81BD20BD0FB6F894FA9AF99A0FBE12BC11BC0895F999FECF5A
S1230AA01FBA81EF91E092BD81BD10BC0FB6F894FA9AF99A0FBEF999FECF1FBA80EF91E0C2
S1230AC092BD81BD8AE080BD0FB6F894FA9AF99A0FBE20915A04F999FECF1FBA82EF91E070
S1230AE092BD81BD20BD0FB6F894FA9AF99A0FBEF999FECF1FBA89E591E092BD81BD84E03B
S1230B0080BD0FB6F894FA9AF99A0FBEF999FECF1FBA81E092E092BD81BD87E180BD0FB64D
S1230B20F894FA9AF99A0FBEF999FECF1FBA82E092E092BD81BD8EE180BD0FB6F894FA9A07
S1230B40F99A0FBEF999FECF1FBA8CE090E092BD81BD85E080BD0FB6F894FA9AF99A0FBEA9
S1230B60F999FECF1FBA8FE691E092BD81BD82E380BD0FB6F894FA9AF99A0FBEF999FECF80
S1230B801FBA81E791E092BD81BD84E180BD0FB6F894FA9AF99A0FBEF999FECF1FBA80E78C
S1230BA091E092BD81BD81E080BD0FB6F894FA9AF99A0FBEF999FECF1FBA84EF91E092BDE5
S1230BC081BD88EC80BD0FB6F894FA9AF99A0FBEF999FECF1FBA85EF91E092BD81BD81E0D2
S1230BE080BD0FB6F894FA9AF99A0FBEF999FECF1FBA86EF91E092BD81BD84E180BD0FB65D
S1230C00F894FA9AF99A0FBEF999FECF1FBA87EF91E092BD81BD8AE580BD0FB6F894FA9A13
S1230C20F99A0FBEF999FECF1FBA88EF91E092BD81BD88EE80BD0FB6F894FA9AF99A0FBEAB
S1230C40F999FECF1FBA89EF91E092BD81BD83E080BD0FB6F894FA9AF99A0FBE209131011A
S1230C6030913201F999FECF1FBA8BEF91E092BD81BD20BD0FB6F894FA9AF99A0FBE2091F9
S1230C80310130913201F999FECF1FBA8CEF91E092BD81BD30BD0FB6F894FA9AF99A0FBE47
S1230CA02091330130913401F999FECF1FBA8DEF91E092BD81BD20BD0FB6F894FA9AF99A4E
S1230CC00FBE2091330130913401F999FECF1FBA8EEF91E092BD81BD30BD0FB6F894FA9AE3
S1230CE0F99A0FBE2091770330917803F999FECF1FBA8FEF91E092BD81BD20BD0FB6F89447
S1230D00FA9AF99A0FBE2091770330917803F999FECF1FBA80E092E092BD81BD30BD0FB62B
S1230D20F894FA9AF99A0FBEF999FECF1FBA87E092E092BD81BD8CED80BD0FB6F894FA9AF6
S1230D40F99A0FBEF999FECF1FBA83E092E092BD81BD86EE80BD0FB6F894FA9AF99A0FBE9F
S1230D608CE192E028ECF999FECF1FBA92BD81BD20BD0FB6F894FA9AF99A0FBE019632E0EC
S1230D808C32930781F7F999FECF1FBA8FE891E092BD81BD82E280BD0FB6F894FA9AF99AB9
S1230DA00FBEF999FECF1FBA86E092E092BD81BD81E080BD0FB6F894FA9AF99A0FBE12BC14
S1230DC011BC08958F929F92AF92BF92CF92DF92EF92FF920F931F93CF93DF93C0E0D0E065
S1230DE035E0832E32E0932E23EDA22E23E0B22EF999FECF92BC81BCF89A60B5F999FECFA3
S1230E00B2BCA1BCF89AE0B46E01CC0CDD1C2FEF31E0C20ED31EF6012081318170E080E0B3
S1230E2090E040E050E00E94292CFF2400E010E0A80197010E94292C24E630E040E050E062
S1230E400E947B2C79018A01C801B70124EF31E040E050E00E94292C28EC30E040E050E0E0
S1230E60E20EF31E041F151FA80197010E947B2CCA01B9012FEF30E040E050E00E94292C92
S1230E8025E030E040E050E00E947B2C82E0220F331F441F551F8A95D1F7CA01B90124E66E
S1230EA030E040E050E00E947B2CF601318320832196C732D10509F09BCFC0E0D0E009EC09
S1230EC0802E03E0902E13EDA12E13E0B12EF999FECF92BC81BCF89A60B5F999FECFB2BCC0
S1230EE0A1BCF89AE0B46E01CC0CDD1C2DE432E0C20ED31EF6012081318170E080E090E0DD
S1230F0040E050E00E94292CFF2400E010E0A80197010E94292C24E630E040E050E00E944F
S1230F207B2C79018A01C801B70124EF31E040E050E00E94292C28EC30E040E050E0E20EB1
S1230F40F31E041F151FA80197010E947B2CCA01B9012FEF30E040E050E00E94292C25E09C
S1230F6030E040E050E00E947B2CA2E0220F331F441F551FAA95D1F7CA01B90124E630E042
S1230F8040E050E00E947B2CF601318320832196C732D10509F09BCFC0E0D0E0FAEC8F2E8A
S1230FA0F3E09F2EE3EDAE2EE3E0BE2EF999FECF92BC81BCF89A60B5F999FECFB2BCA1BC77
S1230FC0F89AE0B46E01CC0CDD1C2BE932E0C20ED31EF6012081318170E080E090E040E036
S1230FE050E00E94292CFF2400E010E0A80197010E94292C24E630E040E050E00E947B2CE8
S123100079018A01C801B70124EF31E040E050E00E94292C28EC30E040E050E0E20EF31E66
S1231020041F151FA80197010E947B2CCA01B9012FEF30E040E050E00E94292C25E030E0BC
S123104040E050E00E947B2C62E0220F331F441F551F6A95D1F7CA01B90124E630E040E0D1
S123106050E00E947B2CF601318320832196C732D10509F09BCFC0E0D0E034E0832E32E095
S1231080932E23EDA22E23E0B22EF999FECF92BC81BCF89A60B5F999FECFB2BCA1BCF89A7B
S12310A0E0B46E01CC0CDD1C29EE32E0C20ED31EF6012081318170E080E090E040E050E0B4
S12310C00E94292CFF2400E010E0A80197010E94292C24E630E040E050E00E947B2C7901BD
S12310E08A01C801B70124EF31E040E050E00E94292C28EC30E040E050E0E20EF31E041FDD
S1231100151FA80197010E947B2CCA01B9012FEF30E040E050E00E94292C25E030E040E0DE
S123112050E00E947B2C82E0220F331F441F551F8A95D1F7CA01B90124E630E040E050E0A0
S12311400E947B2CF601318320832196C732D10509F09BCFDF91CF911F910F91FF90EF90DD
S1231160DF90CF90BF90AF909F908F900895EAE7F0E0108210927C0080E880BF87EE8083B4
S123118011B885E090E09093F4038093F30388E790E09093E8038093E70384E690E09093A3
S12311A0F6038093F5039093FE038093FD0386E490E09093F8038093F70308950F931F93FA
S12311C0CF93DF93282F30E0F901EE0FFF1FEE5FFE4F0081118183E0033F180718F0E2E37D
S12311E0F0E04AC083E00F3D180718F0EAE0F0E043C0A0E0B0E087E290E0289FA001299F85
S1231200500D389F500D1124EA01CA0FDB1FCC0FDD1FC150DE4F888199818017910730F5BA
S1231220FD013197E40FF51FEE0FFF1FE150FE4F208131816081718148815981FD01EE0F80
S1231240FF1FEE0FFF1FEA0FFB1F3596201B310BC901880F991F880F991F641B750B820F04
S1231260931F0E94542CE60FF71F06C01196A732B10551F6E8ECF0E0CF01DF91CF911F9154
S12312800F9108950F931F93CF93DF93AC01E0E0F0E0EF01CC0FDD1FDE01A95CBC4F8D91D4
S12312A09C91119748175907C0F56D917C913197EE0FFF1FDF01A95CBC4F8D919C91119710
S12312C0681B790B8D919C91C15BDC4F28813981E15BFC4F00811181481B590B84E690E0D3
S12312E0DC014A9FC0014B9F900D5A9F900D11240E94542C201B310B0190F081E02D629F68
S1231300C001639F900D729F900D112464E670E00E94542C6E0F7F1F09C03196EA30F1050F
S123132009F0B7CF6091630370916403CB01DF91CF911F910F9108958091E7039091E803DB
S1231340282F205527FF0AC080911401909115019C01220F331F280F391F1FC02F312CF066
S1231360209114013091150118C04091140150911501332727FD309588E290E0821B930BBF
S12313809C01249FC001259F900D349F900D11246AE070E00E94542C9B01C90108950F93C1
S12313A01F93CF93DF93AC0180917A0390917B034817590718F4E0EFF0E057C0809196039E
S12313C0909197038417950718F4E0E0F0E04DC0E1E0F0E0EF01CC0FDD1FDE01A658BC4F2E
S12313E08D919C91119748175907C0F56D917C913197EE0FFF1FDF01A658BC4F8D919C9160
S12314001197681B790B8D919C91E856FC4F20813181C856DC4F08811981481B590B84E655
S123142090E0DC014A9FC0014B9F900D5A9F900D11240E94542C201B310B0190F081E02DB7
S1231440629FC001639F900D729F900D112464E670E00E94542CE61BF70B07C03196EE30D9
S1231460F10509F0B7CFEEEFF0E0CF01DF91CF911F910F9108959C018091E50384FF19C0C7
S1231480C901C2979C0173E0220F331F7A95E1F7880F991F280F391F2455354F442737FD51
S12314A04095542F60E579E784E090E00E949D2C20C08091E50385FD02C024E61AC0C90121
S12314C0C2979C0153E0220F331F5A95E1F7880F991F280F391F2455354F442737FD409546
S12314E0542F60E579E784E090E00E949D2C2C592695822F08950F931F93DF93CF93CDB747
S1231500DEB760970FB6F894DEBF0FBECDBFA89582E50E94402B83E10E94402B80914C0471
S123152090914D04892F0E94402B80914C0490914D040E94402B8091FD039091FE030E94BB
S1231540402B809182040E94402B8091E7039091E8030E94402B8091F5039091F6030E949F
S1231560402B8091F3039091F4030E94402B8091EF039091F0030E94402B80915304909123
S123158054046091180170E00E94542C862F0E94402B80915004909151042091520414E0DB
S12315A0969587951A95E1F7807F822B0E94402B80915004909151040E94402B20915F07A1
S12315C0309160078091EC059091ED058870832B0E94402B80915F07909160070E94402B0B
S12315E0809112060E94402B809181070E94402B8091ED039091EE030E94402B8091EE05E7
S12316009091EF05969587950E94402B8BB18295817089831A828BB18295869581708B8304
S12316201C8280918107992787FD90959E838D8380911206992787FD909598878F83809101
S12316406C0489871A8680916A0490916B049C878B878091F1039091F2039E878D878091BD
S1231660C8039091C903988B8F8780917F04E82FF0E0EE0FFF1F8E010F5F1F4FE00FF11F75
S123168091818295807F892B0E94402B80917F0490E0880F991F080F191FF80180810E941F
S12316A0402B8DEA0E94402B80917F048F5F80937F04883010F010927F0460960FB6F894FB
S12316C0DEBF0FBECDBFCF91DF911F910F9108958F929F92AF92BF92CF92DF92EF92FF928B
S12316E00F931F93CF93DF93A89588E10FB6F89480936000109260000FBE0E94892B882384
S123170011F40C942A130E941D2B90937E0480937D048236910509F478C48336910508F0F2
S12317204BC08D34910509F449C38E34910518F58433910509F44FC78533910570F4883209
S1231740910509F46AC68932910509F490C68132910511F00C942A1355C78534910509F48F
S123176085C18634910509F42CC28134910511F00C942A13BFC08535910509F4D1C586359E
S1231780910568F48235910509F47DC58335910509F4CBC68035910509F05CC7CEC4883535
S12317A0910509F40AC68136910509F451C08735910509F04FC724C58F36910509F414C6EB
S12317C080379105E8F48636910509F4B6C18736910548F48436910509F41DC48536910508
S12317E008F06DC315C48936910509F45AC48D36910509F4A2C28736910509F02BC777C441
S12318008A37910509F44AC48B37910568F48837910509F443C48937910508F052C6803738
S1231820910509F017C7B0C4863F910509F426C2873F910528F4853F910509F00BC79FC186
S1231840873F910569F1883F910509F003C7AFC081E60E94402B80EA0E94402B10927E0430
S123186010927D040EC0E15EF94F80810E94402B80917D0490917E04019690937E0480935A
S12318807D04E0917D04F0917E04E03AF10558F38FEF99E50197F1F7000000C08EE927C0D9
S12318A087EF0E94402B80EA0E94402B10927E0410927D040EC0E154F94F80810E94402B8A
S12318C080917D0490917E04019690937E0480937D04E0917D04F0917E04E03AF10558F3AF
S12318E08FEF99E50197F1F7000000C088E00E94402BB0C610927E0410927D0400E010E0A6
S12319005FEFE52E53EBF52E0E94892B882309F446C0C0917D04D0917E04C03AD10579F50A
S12319200E941D2B90937E0480937D048E3B910579F481E40E94402B81E00E94402B81E073
S12319400E94402B8EEB0E94402B06E11AEF27C081E40E94402B81E00E94402B80E00E9437
S1231960402B8EEB0E94402BC7010197F1F7000000C0E0917B04F0917C04099510C00E9469
S12319801D2BC15ED94F888380917D0490917E04019690937E0480937D0400E010E00F5F66
S12319A01F4F2AEF0030120708F4AECF53C610927E0410927D04C0E0D0E04FEFE42E43EBAC
S12319C0F42E0E94892B882309F449C000917D0410917E04003A110579F50E941D2B9093DA
S12319E07E0480937D048730910579F488EF0E94402B81E00E94402B81E00E94402B87E04C
S1231A000E94402BC6E1DAEF2AC088EF0E94402B81E00E94402B80E00E94402B87E00E94F3
S1231A20402BC7010197F1F7000000C0E0917B04F0917C04099513C000561F4F0E941D2B1F
S1231A40015E194FF801808380917D0490917E04019690937E0480937D04C0E0D0E02196B3
S1231A60FAEFC030DF0708F4ACCFF4C5C0E0D0E038E1F32E0AEF10E00E94892B882309F402
S1231A8055C00E941D2B8A3B910509F0E3C50FB6F894F0926000109260000FBE10927E0421
S1231AA010927D043BC0885B0E94402B8DEF0E94402B80917D0490917E04809FE001819F36
S1231AC0D00D909FD00D112409C0F999FECFD2BDC1BDF89A80B50E94402B219620917D04F2
S1231AE030917E042F5F3F4F209FC001219F900D309F900D112421503040C817D90728F34A
S1231B00822F885B80950E94402B80917D0490917E04019690937E0480937D0480917D0474
S1231B2090917E048430910508F4BDCF21962AEFC030D20708F4A0CF8DC586E60E94402B5D
S1231B4080EA0E94402B10927E0410927D040EC0E455FB4F80810E94402B80917D049091B1
S1231B607E04019690937E0480937D04E0917D04F0917E04E03AF10558F389E9B8CE85EF53
S1231B800E94402B80EA0E94402B10927E0410927D040EC0E45BFA4F80810E94402B809101
S1231BA07D0490917E04019690937E0480937D04E0917D04F0917E04E03AF10558F38AE073
S1231BC096CE10927E0410927D0400E010E02FEFE22E23EBF22E0E94892B882309F446C026
S1231BE0C0917D04D0917E04C03AD10579F50E941D2B90937E0480937D04893B910579F404
S1231C0086E40E94402B81E00E94402B81E00E94402B89EB0E94402B06E11AEF27C086E4AB
S1231C200E94402B81E00E94402B80E00E94402B89EB0E94402BC7010197F1F7000000C02F
S1231C40E0917B04F0917C04099510C00E941D2BC455DB4F888380917D0490917E0401961D
S1231C6090937E0480937D0400E010E00F5F1F4F3AEF0030130708F4AECFECC410927E04BB
S1231C8010927D04C0E0D0E09FEFE92E93EBF92E0E94892B882309F449C000917D041091C9
S1231CA07E04003A110579F50E941D2B90937E0480937D048930910579F486EF0E94402B7F
S1231CC081E00E94402B81E00E94402B89E00E94402BC6E1DAEF2AC086EF0E94402B81E071
S1231CE00E94402B80E00E94402B89E00E94402BC7010197F1F7000000C0E0917B04F09177
S1231D007C04099513C000561F4F0E941D2B04551B4FF801808380917D0490917E04019695
S1231D2090937E0480937D04C0E0D0E02196FAEFC030DF0708F4ACCF8DC48DE60E94402B58
S1231D4089E00E94402B80911F01909120010E94402B80911F0190912001892F0E94402B51
S1231D6080912501909126010E94402B8091250190912601892F0E94402B8091000190915C
S1231D8001010E94402B8091000190910101892F0E94402B809113010E94402B80911201E0
S1231DA00E94402BF999FECF89E591E092BD81BDF89A80B50E94402B82E999CD10927E047E
S1231DC010927D04AA24BB248AE0882E912C0E94892B8A3008F469C00E941D2B90932001EF
S1231DE080931F0100911F01109120010E941D2BD82ECC240C0D1D1D1093200100931F018F
S1231E000E941D2B909326018093250100912501109126010E941D2BF82EEE240E0D1F1D59
S1231E2010932601009325010E941D2B909301018093000100910001109101010E941D2BD9
S1231E40D82FC0E00C0F1D1F10930101009300010E941D2B809313010E941D2B8093120126
S1231E600E941D2BF999FECF1FBA92BC81BC80BD0FB6F894FA9AF99A0FBE0E9422250E94A4
S1231E801D2B823B910561F40E94C704E0917B04F0917C0409950FE6A02E0AEFB02E05C0F3
S1231EA0E0917B04F0917C0409950894A11CB11C20E0A2162AEFB20608F489CFCBC385E693
S1231EC00E94402B83E10E94402B10927E0410927D040EC0EB51FE4F80810E94402B8091C3
S1231EE07D0490917E04019690937E0480937D04E0917D04F0917E04EA30F10558F3809189
S1231F00190190911A016091180170E00E94542C862F0E94402B80911C0190911D016091CB
S1231F20180170E00E94542C862F0E94402B8FEF95E30197F1F7000000C080912A010E943C
S1231F40402B80912B010E94402B80912C010E94402B80912D010E94402B809114019091EA
S1231F60150166E070E00E94542C862F0E94402B809127010E94402BF999FECF8EE691E043
S1231F8092BD81BDF89A80B50E94402B8AE90E94402B8CE60E94402B84E10E94402B1092C9
S1231FA07E0410927D040EC0EE50FA4F80810E94402B80917D0490917E04019690937E04A4
S1231FC080937D04E0917D04F0917E04EA30F10558F310927E0410927D040EC0EE50FA4F7D
S1231FE080890E94402B80917D0490917E04019690937E0480937D04E0917D04F0917E04CD
S1232000EA30F10558F383E972CC0E94A80022C30E94F6001FC381E50E94402B80E10E9498
S1232020402B81E00E94402B82E00E94402B83E00E94402B84E00E94402B85E00E94402B01
S123204086E00E94402B87E00E94402B8091EF039091F0030E94402B80916C040E94402BE3
S123206080916A0490916B040E94402B8091920780950E94402B809182040E94402B8091BF
S123208012060E94402B84E00E94402B85E00E94402B86E00E94402B8EEA29CC0E947B0A2D
S12320A0D9C20E94892B8530E0F30E941D2BC82FD0E00E941D2BC817D90709F0CBC20E9441
S12320C01D2B8C0190937E0480937D040E941D2B0817190709F0BEC20E941D2B863991050D
S12320E009F0B8C280917D04C15ED94F4BC00E94892B8530E0F30E941D2BC82FD0E00E9474
S12321001D2BC817D90709F0A5C20E941D2B8C0190937E0480937D040E941D2B081719077B
S123212009F098C20E941D2B8839910509F092C280917D04C455DB4F25C00E94892B8530F5
S1232140E0F30E941D2BC82FD0E00E941D2BC817D90709F07FC20E941D2B8C0190937E0418
S123216080937D040E941D2B0817190709F072C20E941D2B8F3A910509F06CC280917D046F
S1232180CB5BDE4F888366C2C0E0D0E00E94892B823080F10E941D2B0E941D2B8F389105BB
S12321A009F058C210927E0410927D041CC0EB5BFE4F108180E70E94402B82E00E94402BDE
S12321C080917D040E94402B812F0E94402B8FE80E94402B80917D0490917E04019690932C
S12321E07E0480937D04E0917D04F0917E04E03AF105E8F221963AEFC030D30739F62AC221
S12322000E94892B8530E0F30E941D2BE82ED92E0E941D2BF82E0E941D2B8C0190937E04A9
S123222080937D040E941D2B0817190709F012C28E2D9D2DDF2DC0E08E01080F191F0E945F
S12322401D2B883A9105C9F4C80165E670E00E94FE2BBC01607080917D0490917E04682B99
S1232260792B70937E0460937D04C8014DE650E00E94142C12BC11BCEDC1E0917B04F091F5
S12322807C040995BDCFAA24BB240E94892B833008F43CC00E941D2B082F992E0E941D2B10
S12322A0182F0E941D2B8D3A910509F0D3C1F999FECF802F992DD12ECC24E601C80FD91F86
S12322C0D2BDC1BDF89A90B5F999FECF2196D2BDC1BD2197F89A80B5F82EEE248701090F9C
S12322E0111D84E50E94402B84E00E94402B802F0E94402B8C2F0E94402B8D2F0E94402B78
S1232300812F0E94402B8BEA0E94402B0894A11CB11C80E0A8168AEFB80609F0B6CF9AC126
S1232320AA24BB240E94892B833008F43CC00E941D2B082F992E0E941D2B182F0E941D2BE8
S12323408A3A910509F086C1F999FECF802F992DD12ECC24E601C80FD91FD2BDC1BDF89AC7
S123236090B5F999FECF2196D2BDC1BD2197F89A80B5F82EEE248701090F111D85E50E9460
S1232380402B84E00E94402B802F0E94402B812F0E94402B8C2F0E94402B8D2F0E94402B53
S12323A08AEA0E94402B0894A11CB11CE0E0AE16EAEFBE0609F0B6CF4DC1C0E0D0E00E94D3
S12323C0892B882359F00E941D2B873A910509F041C1E0917B04F0917C0409952196FAEFE6
S12323E0C030DF0761F736C1C0E0D0E00E94892B882369F00E941D2B8039910509F02AC1ED
S12324000E944401E0917B04F0917C04099521962AEFC030D20751F71DC1C0E0D0E00DE640
S123242011E00E94892B8823E1F00E941D2B873D910509F00FC18091F3039091F403F99917
S1232440FECF1FBA12BD01BD80BD0FB6F894FA9AF99A0FBE12BC11BCE0917B04F0917C0437
S1232460099521963AEFC030D307D9F6F3C0C0E0D0E00EE611E00E94892B8823E1F00E94E5
S12324801D2B863D910509F0E5C08091F3039091F403F999FECF1FBA12BD01BD80BD0FB613
S12324A0F894FA9AF99A0FBE12BC11BCE0917B04F0917C04099521968AEFC030D807D9F6A0
S12324C0C9C0C0E0D0E00E94892B823040F10E941D2B892B09F0BEC00E941D2B8638910593
S12324E0F1F489E70E94402B87E00E94402B8FEC0E94402B8FE30E94402B89E00E94402B85
S123250084E50E94402B85ED0E94402B84E10E94402B80E10E94402B86E80E94402B2196B0
S1232520EAEFC030DE0779F695C0C0E0D0E00E94892B823008F448C00E941D2B892B09F032
S123254043C00E941D2B8C3A910509F083C083E50E94402B88E00E94402B8091550490917D
S123256056040E94402B8091550490915604892F0E94402B80911D0690911E060E94402BC0
S123258080911D0690911E06892F0E94402B80911606909117060E94402B80911606909133
S12325A01706892F0E94402B80919507909196070E94402B8091950790919607892F0E94F8
S12325C0402B8CEA0E94402B2196FAEFC030DF0709F0ADCF3FC0C0E0D0E00E94892B8230C7
S12325E058F00E941D2B892BA9F50E941D2B8B3C910511F40E945F0121962AEFC030D2076C
S123260061F728C0C0E0D0E004E610E00E94892B8330D8F00E941D2B0197E1F40E941D2B3A
S1232620FC01E09FC001E19F900DF09F900D112490937A04809379040E941D2B8E3D91055F
S123264021F010927A04109279042196FAEFC030DF07E1F6A895DF91CF911F910F91FF90ED
S1232660EF90DF90CF90BF90AF909F908F900895CF93DF932B9ACFEFD3E224C0CE01019739
S1232680F1F7000000C00E94680B2D982C9ACE010197F1F7000000C081E20E94402B80E00F
S12326A00E94402B8EED0E94402B2D9A2C98289A299A8091790490917A04019790937A040B
S12326C0809379048091790490917A040B97B0F62D9A2C9A10927A0410927904DF91CF9155
S12326E008952F923F924F925F926F927F928F929F92AF92BF92CF92DF92EF92FF920F9359
S12327001F93CF93DF93259A2D9A249A2C9A14BEA89588E10FB6F8948093600010926000E7
S12327200FBE1092600710925F070E948B2A259A249A00002D9A2C9A81E080931C06569AD0
S12327408093F005209A219A219A209A289A299A299A289A549A559A5C9A5D9A229A239A36
S1232760569A2A9A2B985E9800000000529853983B98439A3A98429A3998419A3898409A5F
S12327800E94922AF999FECF8AE591E092BD81BDF89A80B580935B0478940E9422250E943B
S12327A07B2A0E94091C10927A0010927C0080E880BF87EE80937A0011B885E090E0909305
S12327C0F4038093F30388E790E09093E8038093E70384E690E09093F6038093F5039093E7
S12327E0FE038093FD0386E490E09093F8038093F7030E94E2062A9A2B98F999FECF87E0E5
S123280090E092BD81BDF89A80B512BC11BC85FFEEC080910001909101019F7D90930101AD
S1232820809300010E94C7040E944E050E94F6000E94A8000E944401F999FECF1FBA89E5AF
S123284091E092BD81BD82E080BD0FB6F894FA9AF99A0FBEF999FECF1FBA8BE090E092BD30
S123286081BD89E180BD0FB6F894FA9AF99A0FBEF999FECF1FBA8CE090E092BD81BD8EE11A
S123288080BD0FB6F894FA9AF99A0FBEF999FECF1FBA8EE090E092BD81BD8EE180BD0FB69E
S12328A0F894FA9AF99A0FBE80E090E0FC01EB51FE4FE081F999FECF1FBA825A9E4F92BD8D
S12328C081BDE0BD0FB6F894FA9AF99A0FBE8D5591408A30910551F780E090E0FC01E65D79
S12328E0FE4FE081F999FECF1FBA87599E4F92BD81BDE0BD0FB6F894FA9AF99A0FBE8856D4
S123290091408430910551F780E090E0FC01EE50FA4FE081F999FECF1FBA8E589E4F92BD41
S123292081BDE0BD0FB6F894FA9AF99A0FBE815791408A30910551F780E090E0FC01EE5027
S1232940FA4F2089F999FECF1FBA84589E4F92BD81BD20BD0FB6F894FA9AF99A0FBE8B57EF
S123296091408A30910551F720911506F999FECF1FBA81E791E092BD81BD20BD0FB6F89452
S1232980FA9AF99A0FBE2091140130911501F999FECF1FBA8DE090E092BD81BDC90166E0F0
S12329A070E00E94542C60BD0FB6F894FA9AF99A0FBEF999FECF1FBA8DE691E092BD81BD96
S12329C084E180BD0FB6F894FA9AF99A0FBEF999FECF1FBA8EE691E092BD81BD81EE80BDB6
S12329E00FB6F894FA9AF99A0FBE12BC11BC0E942C010E945F010E94C4000E947A0080918F
S1232A0093078E3C24F08091930783337CF010929307F999FECF1FBA8CE094E092BD81BD8C
S1232A2010BC0FB6F894FA9AF99A0FBE8091A0078E3C24F08091A00783337CF01092A007C8
S1232A40F999FECF1FBA8DE094E092BD81BD10BC0FB6F894FA9AF99A0FBE809189078E3C50
S1232A6024F08091890783337CF010928907F999FECF1FBA8EE094E092BD81BD10BC0FB611
S1232A80F894FA9AF99A0FBE809187078E3C24F08091870783337CF010928707F999FECFE5
S1232AA01FBA8FE094E092BD81BD10BC0FB6F894FA9AF99A0FBE809100019091010185FD01
S1232AC007C080916F008B7F80936F002D9A2C9A80912901882311F480E801C080E4809307
S1232AE03B011092E60380911401909115018D5A9D4030F08CEA9DE0909315018093140176
S1232B001092490486B3866086BB78948AEA0E94402B80E00E94402B85E50E94402B86B1BA
S1232B208695817080935D0480916E00836080936E002A9AE89AFF24F394E8EEAE2EE3E0C9
S1232B40BE2E74E0472E66E0362E52E4252E4BE4C42ED12C33E0932E24E4822E94E6E92E4E
S1232B6082E0782E05E4602E11E4512EA89580914C0490914D048B34910548F18091490462
S1232B80882329F580915F07909160079F7E9093600780935F0780916E00836080936E0066
S1232BA02A9A2B9AF092490480915F079091600780629093600780935F0780915F0790913D
S1232BC0600790629093600780935F074AC020914904213009F045C080914C0490914D046B
S1232BE08234910508F03DC080916F008D7F80936F00809170008C7F8093700080916F00F3
S1232C008B7F80936F0080916E00836080936E0080915F07909160078F7D90936007809399
S1232C205F0780915F0790916007877F9093600780935F07289A299A299A289A5C9A5D9A2B
S1232C402D9A2C9A20931C061092490480915F07909160079F7D9093600780935F0710925F
S1232C60470480914904813021F58091E403823028F080916F00856080936F0080916F00B7
S1232C80826080936F008091700083608093700080916E00836080936E0080915F0790916A
S1232CA0600788609093600780935F072A9A2B9A23C01092E403109247042D9A2C9AF092CD
S1232CC01C06289A299A2B98109247041092B3001092540410925304809143019091440196
S1232CE0892B51F42A988091790490917A048536910510F00E94381340914C0450914D0457
S1232D002091250130912601809100019091010180709074822B932B4817590788F4809110
S1232D205F079091600797FD0BC080915F07909160079F7B9093600780935F075F9A0AC063
S1232D4080915F079091600790649093600780935F075F98F89480915504909156048A5A2D
S1232D609A4AB1F080915504909156048555954579F0789480915F079091600780649093B6
S1232D80600780935F07B0923801A09237010AC0789480915F07909160078F7B9093600701
S1232DA080935F07F89480915704909158048A5A9A4AB1F08091570490915804855595451B
S1232DC079F0789480915F079091600780689093600780935F07B0923801A09237010AC0E1
S1232DE0789480915F07909160078F779093600780935F0780913701909138010B9758F02E
S1232E005E9A80913701909138010197909338018093370101C05E988091E603833009F473
S1232E20CAC0843018F4882371F071C0853009F4F7C1853008F422C1863009F4A6C1873038
S1232E4009F076C22EC280914A0490914B048536910508F46FC2E091E603F0E0809178004D
S1232E60909179008C7F65E070E00E94542CEE0FFF1FE95DFB4F718360838091E603C82F7F
S1232E80D0E0E091E603F0E0EE0FFF1FE951FC4F80819181E091E603F0E0EE0FFF1FE95D16
S1232EA0FB4F20813181880F991F880F991F820F931F880F991F6AE070E00E94542CCC0FAA
S1232EC0DD1FC951DC4F7983688310924B0410924A04F092E60350927C000E94680B0E9465
S1232EE09C0990931701809316018091430190914401892B51F080914301909144010197C1
S1232F0090934401809343012A9AA89513C280914A0490914B048536910508F40BC210928D
S1232F204B0410924A04A8958091E603813031F58091080190910901209178003091790098
S1232F40820F931F96958795909309018093080183E00E94DE089093EA038093E90380918F
S1232F60E9039091EA039093FE038093FD03E09285077092E60360927C00DCC18091020114
S1232F80909103012091780030917900820F931F969587959093030180930201D092EC038D
S1232FA0C092EB03D092F803C092F7039092E60380927C00BFC180914A0490914B04853681
S1232FC0910508F4B7C1E091E603F0E080917800909179009695879596958795EE0FFF1FED
S1232FE0E95DFB4F918380838091E603C82FD0E0E091E603F0E0EE0FFF1FE951FC4F8081BA
S12330009181E091E603F0E0EE0FFF1FE95DFB4F20813181880F991F880F991F820F931F91
S1233020880F991F6AE070E00E94542CCB01CC0FDD1FC951DC4F9983888310924B041092DF
S12330404A044092E60380913B0180937C000E94680BA895809169048F5F80936904843095
S123306010F01092690480916904982F917090939F0486958170809318065CC180914A0478
S123308090914B048159914008F454C180912901882329F1E091E603F0E08091780090912C
S12330A079009695879596958795EE0FFF1FE95DFB4F91838083A091E603B0E0E091E6033F
S12330C0F0E0EE0FFF1FE95DFB4F80819181AA0FBB1FA951BC4F11969C938E933EC0E09160
S12330E0E603F0E08091780090917900EE0FFF1FE95DFB4F918380838091E603C82FD0E08D
S1233100E091E603F0E0EE0FFF1FE951FC4F00811181E091E603F0E0EE0FFF1FE95DFB4FF9
S1233120808191810E94CF099C01220F331F280F391FC801F3E0880F991FFA95E1F7801B62
S1233140910B820F931F6AE070E00E94542CCC0FDD1FC951DC4F7983688310924B0410923A
S12331604A0485E08093E60327E420937C0090915D0486B186958170981729F0E0917B04E5
S1233180F0917C040995A895D5C080914A0490914B048536910508F4CDC0E091E603F0E0E7
S12331A080917800909179009695879596958795EE0FFF1FE95DFB4F91838083A091E6037E
S12331C0B0E0E091E603F0E0EE0FFF1FE951FC4F20813181E091E603F0E0EE0FFF1FE95DB3
S12331E0FB4F80819181820F931F880F991F9695879596958795AA0FBB1FA951BC4F11960F
S12332009C938E9310924B0410924A0487E08093E60323E420937C000E94680BA8958AC044
S123322080914A0490914B04893C910508F482C0E091E603F0E08091780090917900EE0FD8
S1233240FF1FE95DFB4F91838083A091E603B0E0E091E603F0E0EE0FFF1FE951FC4F208190
S12332603181E091E603F0E0EE0FFF1FE95DFB4F80819181820F931F96958795AA0FBB1F93
S1233280A951BC4F11969C938E9310924B0410924A043092E60320927C000E94680BA89522
S12332A049C080914A0490914B048536910508F441C0E091E603F0E0809178009091790097
S12332C0969587959695879590E0EE0FFF1FE95DFB4F91838083A091E603B0E0E091E60326
S12332E0F0E0EE0FFF1FE951FC4F20813181E091E603F0E0EE0FFF1FE95DFB4F808191811F
S1233300820F931F96958795AA0FBB1FA951BC4F11969C938E9310924B0410924A0410920D
S1233320E60386E480937C000E94680BA89502C0F092E60380914A0490914B04019690939F
S12333404B0480934A0480914C0490914D048F55914008F443C080919B0787FF02C040E017
S123336002C040919B07809183078F5F809383079091830780918407981790F1109283074B
S12333802091F5033091F603E42FF0E0EF59F84F808190E02817390734F480918107909182
S12333A08207890F12C02091F5033091F603808190E0281739075CF08091810782303CF000
S12333C08091810790918207891B809381078091810785362CF0E092810702C0F092810731
S12333E080914C0490914D048739910508F46DC0809127012091F3033091F40390E0489691
S1233400821793070CF461C08091A8049091A90401969093A9048093A8042091A804309185
S1233420A9048091AA049091AB042817390708F440C01092A9041092A80420914C04309172
S12334404D048091A2049091A3040A972817390730F49091A6048091A704890F15C02091AF
S12334604C0430914D048091A2049091A30449968217930758F49091A6048091A5048917E4
S123348028F48091A60481508093A6049091A6048091A404891718F48091A40408C09091F1
S12334A0A6048091A504981720F48091A5048093A60480914C0490914D048A58924038F4B7
S12334C08091A4048093A60402C01092A6048091E50382FF4EC080914C0490914D04855F25
S12334E0914008F446C080914C0490914D04805D974008F03EC0809127012091F3033091D7
S1233500F40390E00496821793079CF12091F3033091F4038091600490E0019682179307D8
S123352044F18091610490916204A0916304B09164040196A11DB11D8093610490936204F0
S1233540A0936304B09364048091610490916204A0916304B091640481549D40A340B0405F
S123356008F1F0925F0480915F0790916007916015C08091F3039091F4038093600410926C
S1233580610410926204109263041092640410925F0480915F07909160079E7F90936007FC
S12335A080935F07809100019091010192FF27C020914C0430914D04809131019091320137
S12335C082179307E0F420914C0430914D0480913301909134012817390788F480912701FE
S12335E02091F3033091F40390E004968217930734F080915F0790916007946005C080913E
S12336005F07909160079B7F9093600780935F07809100019091010193FF28C0339926C03A
S123362020914C0430914D0480917703909178038217930730F480915F07909160079860FE
S123364005C080915F0790916007977F9093600780935F078091E50383FF27C080914C04C6
S123366090914D04875D964000F115C0809100019091010193FF1FC08091E50383FF15C05E
S123368080918204873588F48091F5039091F6038837910554F48091EC059091ED0588609A
S12336A09093ED058093EC053FC08091EC059091ED05877FF5CF8091EC059091ED05877FF4
S12336C09093ED058093EC0580913A012091F5033091F60390E082179307BCF040914C04AE
S12336E050914D042091210130912201809100019091010180709078822B932B841795070E
S123370050F48091E50380FF06C080915F0790916007986005C080915F0790916007977F52
S12337209093600780935F07809100019091010180FF67C08091300180FF11C080919E0462
S1233740883C28F08091A6048823C9F016C09091A60480919E048695891790F010C08091FA
S1233760300182FF0DC080919E04883C48F080915F079091600796FF02C05C9A01C05C9816
S12337808091300184FF16C080919E04883C28F08091810718165CF12CC0209181078091B1
S12337A09E04332727FD3095869590E0821793070CF11FC08091300186FF1CC080919E0430
S12337C0883CC0F020914C0430914D0480913501909136018217930760F42091F5033091CE
S12337E0F60380915C0490E08217930714F45D9A01C05D9880919E04883C28F010929E0430
S123380002C05C9A5D9A80919E048F5F80939E04ADC91092800081EF9FEF9093890080934A
S1233820880085EF9FEF90938B0080938A0080E88093810080EC9AED909385008093840081
S123384083E090E09093C9038093C8038091C8039091C90380688093810010924D041092EA
S12338604C041CBA80916F00876080936F0010924D0410924C045298539881E080939C0764
S1233880259A249A2D9A2C9A80931C06F999FECF82E092E092BD81BDF89A80B58093B60392
S12338A0F999FECF81E092E092BD81BDF89A80B58093B7038091B7038E3039F08091B70334
S12338C0873119F087E18093B70380915B04813021F480916900836003C08091690082603C
S12338E08093690008951F920F920FB60F9211248F939F9380919C078F5F80939C07809101
S12339009C07882309F449C080915F079091600790619093600780935F071092490480915C
S12339205F07909160079F7D9093600780935F0780916F008B7F80936F0080916F008D7FDE
S123394080936F00809170008C7F8093700080916E00836080936E002D9A2C9A81E08093EE
S12339601C0680915F07909160078F7D9093600780935F0780915F0790916007877F9093EB
S1233980600780935F07289A299A299A289A5C9A5D9A10924D0410924C0478949F918F910B
S12339A00F900FBE0F901F9018951F920F920FB60F9211248F9380912F01813019F482E02C
S12339C08093F1058F910F900FBE0F901F90189580919804882309F47AC040919804809146
S12339E09804823089F42D9A8091570490915804880F991F909358048093570480915704A0
S1233A009091580481600BC080919804803269F42C9A8091570490915804880F991F90939C
S1233A205804809357041092980480918400909185009093A1048093A00481E08093F00557
S1233A408091160690911706892BF1F0809197078823D1F0209116063091170680919507EF
S1233A60909196072817390738F480919507909196078C599F4F04C080911606909117066C
S1233A8090938B0080938A0080914C0490914D048C5D954008F059C08091E50381FF55C0A7
S1233AA080918A0090918B0088539F4F90938B0080938A004093970780918A0090918B00EF
S1233AC08C509E4F90939607809395070895809197078823D1F1209197072230D9F42D98BE
S1233AE08091550490915604880F991F9093560480935504809155049091560481609093BC
S1233B00560480935504209398048091990790919A0715C0209197072032A9F42C98809131
S1233B20550490915604880F991F90935604809355042093980480918B0790918C079093AC
S1233B408B0080938A001092970708951F920F920FB60F9211242F933F934F935F936F9305
S1233B607F938F939F93AF93BF93EF93FF930E94E81C2A9A7894FF91EF91BF91AF919F91ED
S1233B808F917F916F915F914F913F912F910F900FBE0F901F901895282F80915F0790913B
S1233BA0600793FD08C0223019F0203221F402C02D9808952C9808951F920F920FB60F9243
S1233BC011248F939F93F89480918F07882309F486C080916A0490916B0497FD80C0809143
S1233BE0130180958093920780919207909112068C59891B809392079091F105943029F1DF
S1233C00953040F4923051F19330B8F4913009F058C009C09731C1F1933609F441C09E308A
S1233C2009F04FC023C0809192078093B20084E08093B100289883E050C08091920786BDDE
S1233C4083E085BD299884E048C0809192078093B2009093B100289882E03FC08091920780
S1233C6086BD83E085BD299881E037C081E08093CD03809192078093B20084E08093B10064
S1233C802898289887E129C081E08093CE038091920786BD83E085BD299829988EE01DC0AB
S1233CA081E08093CD03809192078093B20084E08093B10028982898299829989093F1050A
S1233CC00EC0809192078093B20084E08093B100289828982998299883E68093F1057894FB
S1233CE09F918F910F900FBE0F901F901895EF92FF920F931F93CF93DF93EC0180915A0473
S1233D00E7E0F0E0E81BF109EE0FFF1FE951FC4F0190F081E02D80915904E81BF109F7FFFB
S1233D2002C0E0E0F0E080912E0126E0829FC00111249C012E9FC0012F9F900D3E9F900DC0
S1233D40112464E670E00E94682CCB01603A71050CF08FE980939807809198076AE00E94BC
S1233D60482C80938A0780918A0780311CF08FE080938A0780914C0490914D04885E934029
S1233D8008F0AAC0109286078FEF80939B0780918A0724E18202C0011124909351048093AF
S1233DA0500480914C0490914D0464E670E00E94542C65506093940780914C0490914D0406
S1233DC0845F914060F410929407E0919407FF27E7FDF095E25CFE4F808190E0A9C0809189
S1233DE094078430E1F5E0915004F0915104E15EF94F2081E0919407FF27E7FDF095E25CFE
S1233E00FE4F6081E0919407FF27E7FDF095E25CFE4F808190E09093EF058093EE05E0914B
S1233E20EE05F091EF0580914C0490914D044091940730E0220F331F261B3109845F914015
S1233E406CE94602A0011124840F951FAC01249FC001259F900D349F900D11243AC0E09102
S1233E609407FF27E7FDF095E15CFE4F6081E0919407FF27E7FDF095E25CFE4F4081E09151
S1233E809407FF27E7FDF095E25CFE4F808190E09093EF058093EE05E091EE05F091EF0502
S1233EA080914C0490914D042091940770E0641B7109845F91404CE9240290011124820F30
S1233EC0931F9C01629FC001639F900D729F900D112464E670E0D1C080914C0490914D044D
S1233EE0875F924250F187EC80938607809186076AE00E94482C80939B0780918A072091AA
S1233F009B0744E18402C0011124332727FD3095820F931F9093510480935004E091500430
S1233F20F0915104E15EF94F808190E0880F991F9093EF058093EE05A8C080914C04909159
S1233F404D04885E934062E370E00E94542C60938607809186076AE00E94482C80939B0769
S1233F6080918A0720919B0744E18402C0011124332727FD3095820F931F90935104809396
S1233F805004E0915004F0915104E15EF94F808190E0880F991F9093EF058093EE058091B9
S1233FA09B0787FD37C080919B0783319CF5E0915004F0915104E05EF94F4081E091500441
S1233FC0F0915104E15EF94F6081E091EE05F091EF053091860780919B0726EF8202C0016B
S1233FE01124830F911D880F991F50E0461B51099C01249FC001259F900D349F900D1124E7
S12340006AE070E00E94682CE60FF71FF093EF05E093EE0580918A0787FD37C080918A0725
S12340208F309CF5E0915004F0915104ED5CF94F4081E0915004F0915104E15EF94F60813C
S1234040E091EE05F091EF053091980780918A0726EF8202C0011124830F911D880F991F63
S123406050E0461B51099C01249FC001259F900D349F900D11246AE070E00E94682CE60F65
S1234080F71FF093EF05E093EE0580914C0490914D04855F914010F46AEB66C080914C04C1
S12340A090914D048952934210F06DE05DC080914C0490914D0485569941B0F080914C04E7
S12340C090914D04845699416AE070E00E94542CCB01880F991F880F991F860F971F64E6FB
S12340E070E00E94542C40C080914C0490914D04815A9F40B0F080914C0490914D04805A70
S12341009F406AE070E00E94542CCB01B3E0880F991FBA95E1F764E670E00E94542C6451BA
S123412023C080914C0490914D04855F914010F460E01AC080914C0490914D04845F91406B
S12341406AE070E00E94542CCB019B01A3E0220F331FAA95E1F7880F991F820F931F64E63E
S123416070E00E94542C67532091EE053091EF05862F992787FD9095820F931F97FF06C0F9
S12341808091EE059091EF0561E0681B40918204445645310CF044E12091EE053091EF055D
S12341A0809112019091480420583040280F311D291B3109842F4C3E0CF48CEE992787FD84
S12341C09095280F391F862F992787FD9095280F391F309381042093800480919F07882399
S12341E039F020918004309181048091930706C020918004309181048091A007992787FD2F
S12342009095820F931F90938104809380048091800490918104895592403CF0E8E5EE2EF3
S1234220E2E0FE2E012D112D15C08091800490918104059734F475E0E72EF12C012D112D59
S123424009C080918004909181047C010027F7FC0095102F20914E0430914F042C0F3D1F3D
S123426040E050E0C801B7010E94292C28E037E040E050E00E947B2C790180919F079E01EA
S12342802E193F09882329F030939A072093990704C030938C0720938B079E012E193F0983
S12342A0C901DF91CF911F910F91FF90EF900895EF92FF920F931F93CF93DF93EC0160914D
S12342C09B0470919C042091130126952695620F711D7695679580E090E02AE530E040E04A
S12342E050E00E94292C20914E0430914F042C0F3D1FE3E036952795EA95E1F740E050E0F4
S12343000E949D2CB901CA01E0919B07FF27E7FDF095E854FC4FE08124EB30E02E1B31097D
S1234320442737FD4095542F620F731F841F951F9E0140E050E00E94292C22E130E040E00F
S123434050E00E949D2CCA01B9012AE030E040E050E00E949D2C79018A012A97CE01A0E04F
S1234360B0E02A968E159F05A007B1071CF42AE030E003C09E012E193F09C901DF91CF918E
S12343801F910F91FF90EF9008950F931F93CF93DF9380918400909185009093A2078093DC
S12343A0A1078091840090918500C29708F41EC380919C07882349F088EE9DEF9093CC0354
S12343C08093CB0310929C0760C080918400909185006091CB037091CC039B0136952795A6
S12343E0AB01F3E056954795FA95E1F7241B350B8217930790F481E080939F078091E403C4
S12344008F5F8093E40380912F01823009F0EEC28091B7038093F105E9C280914C04909113
S12344204D04E0914E04F0914F0420918400309185008091B60390E0261B370BAC01429FCA
S1234440C001439F900D529F900D11246EE170E00E94682CCB018E0F9F1F62E070E00E9425
S1234460682C70934F0460934E0410924F0410924E0480918400909185009093CC038093E0
S1234480CB0310928500109284008091E403853618F084E68093E40380914704893628F4A7
S12344A0809147048F5F8093470480914C0490914D048C5D954040F42D9B02C02C9904C078
S12344C02D9A2C9A109298041092F00580914C0490914D04C091CB03D091CC03D0931E06CD
S12344E0C0931D0620911D0630911E060091C8031091C90340E050E060E070E489E191E001
S12345000E949D2CCA01B9012EE130E040E050E00E94292C20EC30E0A901049F9001059FA3
S1234520300D149F300D11242050324040E050E00E947B2C30934D0420934C0420918F043F
S12345403091900440918D0450918E04C901880F991F820F931F840F951F96958795969518
S123456087959093900480938F0480918B0490918C0490938E0480938D0480918904909155
S12345808A0490938C0480938B04809187049091880490938A0480938904809185049091DF
S12345A0860490938804809387048091830490918404909386048093850480914C04909114
S12345C04D04909384048093830480914C0490914D048D5D9540D8F04091820480918304F8
S12345E09091840420918F0430919004821B930B23E0429FA0011124840F951F64E09695CA
S123460087956A95E1F7855B809382040FC084E68093820480914E0490914F0464E070E0ED
S12346200E94682C70934F0460934E0410929C0780914C0490914D048C529140A0F5809138
S1234640C8039091C903039771F580919F07882351F584E090E09093C9038093C803809144
S1234660C8039091C903806880938100809184009091850096958795969587959093850091
S123468080938400D695C795D695C795D093CC03C093CB0380911D0690911E0696958795DE
S12346A0969587953AC080914C0490914D0481599140B8F18091C8039091C903049789F5AC
S12346C080919F07882369F583E090E09093C9038093C8038091C8039091C90380688093B2
S12346E081008091840090918500880F991F880F991F9093850080938400CC0FDD1FCC0F6B
S1234700DD1FD093CC03C093CB0380911D0690911E06880F991F880F991F90931E068093D5
S12347201D0680911D0690911E060E94771E90939607809395072091990730919A0780916F
S12347408B0790918C078217930728F48091990790919A0704C080918B0790918C0790930F
S123476096078093950780914C0490914D048A58924038F08091E7039091E8038E369105D9
S12347803CF48CE291E090939E0780939D0704C010929E0710929D078091950790919607CB
S12347A0209116013091170140919D0750919E07821B930B841B950B90939107809390077A
S12347C0809190079091910797FF20C0809190079091910720911D0630911E064091950777
S12347E050919607820F931F8417950778F4809195079091960720911D0630911E06449653
S1234800821B930B9093910780939007F89480914C0490914D04805E9E4208F0B2C080915C
S12348205F079091600793FDACC0809190079091910785369105CCF11092980480914C047C
S123484090914D048855924090F42091950730919607809195079091960796958795969527
S12348608795281B390B3093910720939007809190079091910790938B0080938A0080912F
S12348808A0090918B00909317068093160680919F07882311F480E201C082E080939707D2
S12348A01092980484E090E060C080919007909191078B5B9F4F2CF11092980484E690E058
S12348C090938B0080938A00909317068093160680919F07882329F480E2809397072C98C4
S12348E004C082E0809397072D981092980488E290E090931A068093190684E18093CA0346
S123490038C080911D0690911E062091900730919107280F391F3093170620931606809132
S12349209F07882371F480918B0790918C0790938B0080938A002C9880E28093980482E0E4
S12349400DC08091990790919A0790938B0080938A002D9882E08093980480E280939707DF
S123496084E18093CA0384EB90E090931A068093190610929F0780915F07909160079F773D
S12349800FC080911D0690911E068C509E4F90938B0080938A0080915F07909160079068C0
S12349A09093600780935F0780914C0490914D048D5A9D4070F020911D0630911E06369575
S12349C0279536952795C901880F991F820F931F06C080911D0690911E060E9458219093B7
S12349E089008093880081E080938F077894DF91CF911F910F9108951F920F920FB60F9204
S1234A0011242F933F934F935F936F937F938F939F93AF93BF93EF93FF930E94C5212A9A99
S1234A207894FF91EF91BF91AF919F918F917F916F915F914F913F912F910F900FBE0F90FB
S1234A401F90189521EB30E0F90110821092B6001092B2001092B300A0E7B0E08C91836036
S1234A608C93209A219A219A209A289A299A299A289AEFE6F0E080818D7F80838C918C7F42
S1234A808C9386E0F901808384E6809312060895813099F4289A289A80912F01843021F492
S1234AA0299A299A1092CE031092A6071092A5071092CD031092B1000895823049F4299A48
S1234AC0299A1092A4071092A3071092CE0315BC08951F920F920FB60F9211242F933F9314
S1234AE04F935F936F937F938F939F93AF93BF93EF93FF93F8948091CD03843019F481E03F
S1234B000E9448257894FF91EF91BF91AF919F918F917F916F915F914F913F912F910F9077
S1234B200FBE0F901F9018950F931F938091E7039091E8030A9714F487E003C080915F0407
S1234B4086E08093B1001092B20080914C0490914D04845F914018F41092940716C080911C
S1234B604C0490914D048D56974020F08EE0809394070BC080914C0490914D0464E670E051
S1234B800E94542C655060939407E0919407F0E0E151FE4F80818093130180915F0488230A
S1234BA029F02091C0048091180109C0E0915004F0915104E455FB4F808120911801829F66
S1234BC0C001112490939C0480939B0480914C0490914D04825C914060F58091000190915C
S1234BE0010182FF1CC080919B0490919C042091190130911A01820F931F90939C04809321
S1234C009B0480915F079091600784609093600780935F0780911B0180939A0444C0809118
S1234C205F07909160078B7F9093600780935F073AC080915F07909160078B7F90936007E8
S1234C4080935F0780919A04823068F180919A04815080939A0420919B0430919C0440916A
S1234C60190150911A01E0911901F0911A0180911B0170919A0460911B01240F351F90E023
S1234C80871B9109AC014E9FC0014F9F900D5E9F900D112470E00E94542C261B370B309367
S1234CA09C0420939B0480915F04882309F0E8C080919B0787FD3FC080919B078331DCF5D0
S1234CC0E0915004F0915104E355FB4F4081E0915004F0915104E455FB4F208100919B0403
S1234CE010919C043091860780919B07E091180150E0421B510926EF8202C0011124830FDC
S1234D00911D9C01429FC001439F900D529F900D11246AE070E00E94682CF0E06E9FC001F2
S1234D206F9F900D7E9F900D1124800F911F90939C0480939B0480918A0787FD3FC08091EB
S1234D408A078F30DCF5E0915004F0915104E054FB4F4081E0915004F0915104E455FB4F36
S1234D60208100919B0410919C043091980780918A07E091180150E0421B510926EF820211
S1234D80C0011124830F911D9C01429FC001439F900D529F900D11246AE070E00E94682C88
S1234DA0F0E06E9FC0016F9F900D7E9F900D1124800F911F90939C0480939B0480910001F1
S1234DC09091010184FF5CC020911304309114048091F3039091F40328173907FCF48091CD
S1234DE0F3039091F4032091130430911404821B930B64E070E00E94682C809152048617F7
S1234E0010F460935204809152048A3018F089E0809352048091280180939D0430919D04F6
S1234E203430C8F080919B0490919C04E0915204F0E0EB51FE4F2081820F911D90939C041E
S1234E4080939B04315030939D0480915F0790916007806109C01092520410929D048091C2
S1234E605F07909160078F7E9093600780935F078091F3039091F4039093140480931304AC
S1234E80809100019091010191FD09C08091E50386FF94C080915F04882309F48FC0809134
S1234EA014068F5F809314069091140680911506981708F486C0109214068091EF03909181
S1234EC0F003E0918A07FF27E7FDF095EE50FA4F208130E02817390734F480911206909121
S1234EE01306890F19C08091EF039091F003E0918A07FF27E7FDF095EE50FA4F208130E044
S1234F00821793075CF48091120618163CF48091120690911306891B8093120680915F07DA
S1234F20909160079D7F9093600780935F0720911206E0918A07FF27E7FDF095EE50FA4FE5
S1234F408089332727FD309590E08C599F4F8217930754F4E0918A07FF27E7FDF095EE5074
S1234F60FA4F80898C591EC020911206E0918A07FF27E7FDF095EE50FA4F4089332727FDF0
S1234F80309584E690E0841B910928173907CCF4E0918A07FF27E7FDF095EE50FA4F9089C5
S1234FA084E6891B8093120680915F079091600792609093600780935F0703C084E6809380
S1234FC0120680919B0490919C042091850730E062E070E00E94682C269FC001279F900D46
S1234FE0369F900D112464E670E00E94542C660F771F70939C0460939B0480911E01209129
S1235000FD033091FE0390E0C196821793070CF451C0809100019091010181FF4BC08091EE
S1235020FD039091FE03C397F4F020911C0130911D0140911C0150911D018091FD03909140
S1235040FE0360911E0170E06E5C7F4FFC01E49FC001E59F900DF49F900D11240E94542C6A
S1235060261B30E004C020911C0130911D0180919B0490919C04280F391F30939C04209354
S12350809B04309B05C0809123019091240104C080911F01909120019093220180932101B0
S12350A080915F079091600782609093600780935F0711C080915F07909160078D7F909309
S12350C0600780935F0780911F019091200190932201809321018091EC059091ED0583FF67
S12350E01CC0E0919B04F0919C0420913D0180919B0490919C0464E170E00E94682C30E064
S1235100629FC001639F900D729F900D11248E0F9F1F90939C0480939B0480910001909144
S1235120010190FF4DC08091E7039091E803823891050CF045C080919B0490919C04209153
S12351402A01820F911D90939C0480939B04E091E703F091E8036091180120912A0182E855
S123516090E08E1B9F0B70E0AB01849FB001859F700D949F700D11248FEF90E0FB01E89FA1
S1235180B001E99F700DF89F700D1124882777FD8095982F30E040E050E00E94292C20E4B2
S12351A03FE140E050E00E947B2CC90120919B0430919C04280F391F30939C0420939B0473
S12351C020919B0430919C048091180145EF849FC00111248217930754F480911801849FDB
S12351E0C001112490939C0480939B040BC080919B0490919C041816190624F010929C0461
S123520010929B0480919B0490919C04909354048093530478941F910F9108951F920F92A8
S12352200FB60F9211242F933F934F935F936F937F938F939F93AF93BF93EF93FF93F894CB
S12352402091CD03223039F0243009F44FC0213009F051C01CC08091A5079091A6078F3F5E
S12352609105D1F1C8F18091A5079091A6078F5F8093B3008091A5079091A6078F5F904091
S12352809093A6078093A5072093CD0334C00E94942580915304909154049093A6078093E5
S12352A0A5078091A5079091A6078F3F9105A1F098F08091A5079091A6078F5F8093B300F7
S12352C08091A5079091A6078F5F90409093A6078093A50782E007C08091A5079091A6073E
S12352E08093B30084E08093CD0305C081E00E9448251092CD037894FF91EF91BF91AF914A
S12353009F918F917F916F915F914F913F912F910F900FBE0F901F9018951F920F920FB64B
S12353200F9211242F933F934F935F936F937F938F939F93AF93BF93EF93FF93F89480917E
S12353402F01843008F05EC02091CE03223039F0243009F453C0213009F083C020C0809170
S1235360A3079091A4078F3F910591F088F08091A3079091A4078F5F87BD8091A3079091C1
S1235380A4078F5F90409093A4078093A30733C08091A3079091A40787BD84E024C08091FE
S12353A05304909154049093A4078093A30724E025BD16BC8091A3079091A4078F3F9105EB
S12353C0A9F0A0F08091A3079091A4078F5F87BD8091A3079091A4078F5F90409093A407D4
S12353E08093A30782E08093CE033BC08091A3079091A40787BD2093CE0333C082E00E9465
S123540048252FC08091300181FD04C08091300185FF24C084E085BDE0915004F0915104BD
S1235420EB5BFE4F80818C5E87BD80915F079091600797FD16C080915F079091600792FDAF
S123544010C087B58F3168F08091300181FD5C988091300185FF05C05D9803C016BC81E0FA
S123546087BD7894FF91EF91BF91AF919F918F917F916F915F914F913F912F910F900FBE0C
S12354800F901F9018951F920F920FB60F9211242F933F934F935F936F937F938F939F9350
S12354A0AF93BF93EF93FF93F89480912F01843040F48091CE03843061F482E00E9448252F
S12354C008C08091300181FD5C9A8091300185FD5D9A7894FF91EF91BF91AF919F918F9193
S12354E07F916F915F914F913F912F910F900FBE0F901F901895549A559A5C9A5D9A15BC36
S1235500EEE6F0E080818360808384E085BD16BC82E187BD089511B88FEF84B915B887B9AF
S12355208AB9089588E98093C1001092C50083E18093C4008EEE97E09093AC078093AB0712
S12355409093A8078093A7078EEA97E09093AA078093A90790932F0880932E081092AD0735
S123556010921B0608951F920F920FB60F9211248F939F93EF93FF938091AD07882311F100
S1235580E091AB07F091AC0781918093C600F093AC07E093AB07EE52F84030F08EEE97E0DF
S12355A09093AC078093AB078091AD0781508093AD078091AD07882329F48091C1008F7D84
S12355C08093C100FF91EF919F918F910F900FBE0F901F9018951F920F920FB60F9211243F
S12355E02F938F939F93EF93FF938091C600E0912E08F0912F08808380911B068F5F809311
S12356001B0680912E0890912F08019690932F0880932E088E5E974030F08EEA97E0909397
S12356202F0880932E08FF91EF919F918F912F910F900FBE0F901F90189580911B06882382
S123564019F42FEF3FEF1AC0F89480911B06815080931B06E091A907F091AA072191F093C8
S1235660AA07E093A907EE5EF74030F08EEA97E09093AA078093A907789430E0C9010895A6
S1235680982F8091AD078F33E0F78091AD07803410F080E00895F8948091AD078F5F809319
S12356A0AD07E091A707F091A80790838091A7079091A80701969093A8078093A7078E5237
S12356C0984030F08EEE97E09093A8078093A7078091C10080628093C100789481E00895B6
S12356E0CF93DF93EC0104C00E94402B8111219688818823C9F781E0DF91CF9108958FEC0E
S123570093E00E94702B089587ED93E00E94702B089580911B0608959F92AF92BF92CF9284
S1235720DF92EF92FF920F931F93DF93CF93CDB7DEB729970FB6F894DEBF0FBECDBF7C011D
S1235740062FDE011196EAEDF3E089E001900D928150E1F719E099E0A92EB12C6E0108946D
S1235760C11CD11C8CE2982E002371F09501211B3109802F90E02817390730F01150F60181
S1235780E10FF11D908200E01150F601E10FF11DC7016AE070E00E94542C805D8083C70193
S12357A06AE070E00E94542C7B016115710511F4002311F00630C0F219E0141B7E0108946D
S12357C0E11CF11C07C0F701E10FF11D80810E94402B1F5F1930B8F329960FB6F894DEBFD1
S12357E00FBECDBFCF91DF911F910F91FF90EF90DF90CF90BF90AF909F900895DF92EF9204
S1235800FF920F931F937B018C01FB010995D82EC8010196F7010995982F8D2D1F910F912F
S1235820FF90EF90DF900895DF92EF92FF920F931F93D72E7A018C01FA010995C80101966D
S12358406D2DF70109951F910F91FF90EF90DF900895629FD001739FF001829FE00DF11DB9
S1235860649FE00DF11D929FF00D839FF00D749FF00D659FF00D9927729FB00DE11DF91F24
S1235880639FB00DE11DF91FBD01CF0111240895991B79E004C0991F961708F0961B881F49
S12358A07A95C9F780950895AA1BBB1B51E107C0AA1FBB1FA617B70710F0A61BB70B881F87
S12358C0991F5A95A9F780959095BC01CD01089597FB092E07260AD077FD04D0E5DF06D069
S12358E000201AF4709561957F4F0895F6F7909581959F4F0895A1E21A2EAA1BBB1BFD01F9
S12359000DC0AA1FBB1FEE1FFF1FA217B307E407F50720F0A21BB30BE40BF50B661F771FF9
S1235920881F991F1A9469F760957095809590959B01AC01BD01CF01089597FB092E05265A
S12359400ED057FD04D0D7DF0AD0001C38F450954095309521953F4F4F4F5F4F0895F6F7CC
S123596090958095709561957F4F8F4F9F4F0895F894FFCF2F00010002000300040005001F
S12359800600070008003228E80390010614001E1E003C581B581B88136419121E01010254
S12359A003040A0411C4098813C4096400DCE64003020A14324696500000000000000000A1
S12359C00000000000000000000000000000000000000000000000000000000000000000C3
S12359E0000000000000000000000000000000000000000000000000000102030405060787
S1235A0008090A0B0C0D0E0F100102030405060708090A0B0C0D0E0F100102030405060772
S1235A2008090A0B0C0D0E0F1014161718191A1B1C1D1E1F2021222324191A1B1C1D1E1F6B
S1235A402021222324252627271E1F2022232425262728292A2B2C2D2E0002040607080976
S1235A600A0C0E28262422201E1E1E1E1E1E1E1E1E1E1EF0FF80BBE0880465484BA4380294
S1235A802BF0207019CC13860F440CC209D0074C061B052A046A03D1025602F201A1015FAC
S1235AA0012801FB00D600B7009D0087007500660059004D0044003C0034002E002900255B
S1235AC000F0FF80BBE0880465484BA438022BF0207019CC13860F440CC209D0074C061BBF
S1235AE0052A046A03D1025602F201A1015F012801FB00D600B7009D0087007500660059D9
S1235B00004D0044003C0034002E0029002500F0FF80BBE0880465484BA438022BF02070ED
S1235B2019CC13860F440CC209D0074C061B052A046A03D1025602F201A1015F012801FB91
S1235B4000D600B7009D0087007500660059004D0044003C0034002E0029002500F0FF8070
S1235B60BBE0880465484BA438022BF0207019CC13860F440CC209D0074C061B052A046AF0
S1235B8003D1025602F201A1015F012801FB00D600B7009D0087007500660059004D004444
S1235BA0003C0034002E00290025000000F5047E05AE066C08C00AB30D630F8B10D711884A
S1235BC013000000000A000F001E003C007800FA007201E00180028002000008000A000C53
S1235BE0000E00C80A4A067E048403AC0D641A002000270032003E0066008E00B202EB02E5
S1235C00240337034B03560361037003E800D600C200B0009D008A007800780065005200A3
S1235C2040002D0019000700000001175A5A5A505050505050505050505050500300320068
S11B5C40FA04041B5B481B5B324A000D0A00202020202020202020005F
S50302E317
